:020000020000FC
:1000000022C060C35FC35EC35DC35CC35BC35AC32E
:100010003EC34FC357C356C355C354C3E9C252C3AB
:1000200051C350C34FC3ED05E3C70FCEEE85EFCFED
:100030000002AF64EA2212FA1C38F031117A103053
:10004000FFFD509B15DD04E00EBF0FE50DBF02E084
:1000500004BB01E405BB0FEF07BB01BB002708BBD6
:1000600002BB0093740000936C0000936D0000933A
:1000700068000093690000936A0000936B0000938E
:100080006E0000936F000AE0009377000093000079
:10009000009300000093000000937B000093000099
:1000A00000930000009300002224332403E003BFE8
:1000B00003E00EBD05E009BF0EE806B9002702BF48
:1000C0000DBD0CBD53D2BCD174D27894FAD104D0FA
:1000D0003BD0D7D030D2FACF03E0302E989B0CC063
:1000E0000895CFD0989BFDCF00917300013011F09F
:1000F000A998C8C1DDD1C6C1C4D0032D003089F391
:10010000989BFACF00917300003039F0013049F02C
:10011000023019F0033099F0089501E00093730064
:10012000089502E00093730000916E0010916F003B
:1001300000937F0010938000AFD13AD1089502E080
:1001400000937300A998089523D2013031F00091F3
:1001500068001091690037D008C000916A001091C2
:100160006B0031D0203009F42AE020937E001093F8
:100170007D0000937C000DE000937B0000917300F4
:10018000013029F000916C0010916D0007C0022D24
:10019000003079F000916E0010916F0014D0209320
:1001A0007A0010937900009378000CE000937700B8
:1001B00008950AE000937A00009379000093780094
:1001C00000937700089504561040F8F0045610404C
:1001D000F0F004561040E8F004561040E0F00456E9
:1001E0001040D8F004561040D0F004561040C8F02B
:1001F00004561040C0F004561040B8F004561040A9
:10020000B0F02BE01BE00BE0089520E011C021E0EE
:100210000FC022E00DC023E00BC024E009C025E0A0
:1002200007C026E005C027E003C028E001C029E0A0
:100230000C590A5098F00A5098F00A5098F00A5059
:1002400098F00A5098F00A5098F00A5098F00A5026
:1002500098F00A5098F00A5019E011C010E00FC051
:1002600011E00DC012E00BC013E009C014E007C09C
:1002700015E005C016E003C017E001C018E0065FF6
:10028000089500917600003019F100917E0088D029
:1002900002BBAED0C0988CD000917D0081D0C09AB6
:1002A00002BBACD0C19884D000917C0079D0C19AB7
:1002B00002BBC2987DD000917B0072D0C29A02BB73
:1002C000C39876D0C39A00917500003019F141C0EF
:1002D00000917E005DD002BB76D0C09A69D00091BB
:1002E0007D0056D0C09802BB74D0C19A61D00091F5
:1002F0007C004ED0C19802BBC29A5AD000917B00BC
:1003000047D0C29802BBC39A53D0C39800917500DE
:100310000130F9F000917A003BD002BB9498C69A64
:1003200047D00091790034D0C69802BBC79A40D01C
:10033000009178002DD0C79802BBC49A39D00091A3
:10034000770026D0C49802BB4AD0C59A31D0C59850
:10035000089500917A0024D002BB949AC69828D0C0
:10036000009179001DD0C69A02BBC79821D0009198
:10037000780016D0C79A02BBC4981AD000917700B3
:100380000FD0C49A02BB40D0C59812D0C59A089528
:10039000E6E3F0E020E0E00FF21FC895002D08959D
:1003A000E6E2F0E020E0E00FF21FC895002D08958E
:1003B0001F932F9312E324E11A95F1F72A95E1F7A1
:1003C0002F911F91089500917400013009F09498C5
:1003D0000895009174000030D9F394980895009125
:1003E0007300023021F4022D003009F09498089532
:1003F00000917400013009F0949A089500917400FE
:100400000030D9F3949A089500917300023021F4DA
:10041000022D003009F0949A0895E199FECF222729
:100420001EBB2FBBE09A0DB30895E199FECFF8945F
:1004300022271EBB2FBB0DBBE29AE19A7894089548
:1004400017E3EBDF0434A9F41AE0E7DF009371004F
:100450001BE0E3DF009370001CE0DFDF009373001C
:100460001DE0DBDF009380001EE0D7DF00937F00FC
:10047000089517E304E4D9DF1AE00027D6DF1BE074
:100480000027D3DF1CE00027D0DF1DE00027CDDFF1
:100490001EE00027CADFD7CD1CE002E0C6DF1DE06A
:1004A00000918000C2DF1EE000917F00BEDF089552
:1004B0001AE000916D00B9DF1BE000916C00B5DF20
:1004C000089500917200073461F500916200109167
:1004D00063002BD000936A0010936B0000916000C2
:1004E0001091610022D00093680010936900009180
:1004F00064001091650019D0209170003091710056
:10050000021B130B78F000936C0010936D000091A8
:1005100066001091670009D000936E0010936F0081
:1005200048D0089500271127EECF24E016950795AF
:100530002A95E1F7089500917300025078F0009138
:100540007300033089F000917F00109180002091AA
:100550006C0030916D00021B130B10F0A9980895E8
:100560000091030000937300A99A0895002707BB28
:1005700008BB979A1DDF00E0B39901E00093760075
:1005800000E0B59901E0009375000FEF07BB0895F7
:1005900000916A0010916B0024E63327021B130BB5
:1005A00020F001E000937400089500270093740088
:1005B000089504E007B900270093720000936600D5
:1005C0000093670000936000009361000093620055
:1005D000009363000093640000936500089505E0B4
:1005E00007B94FC003E007B94CC002E007B949C0E2
:1005F0009FB70F931F932F933F9324B135B1009171
:1006000072000734F1F1039500937200013139F360
:10061000033241F3053349F3015198F00091720020
:100620000352D0F000917200055308F1009166006A
:1006300010916700200F311F2093660030936700F0
:1006400020C00091600010916100200F311F2093A5
:1006500060003093610015C000916200109163004A
:10066000200F311F20936200309363000AC0009175
:10067000640010916500200F311F209364003093B7
:1006800065003F912F911F910F919FBF18959FB7C4
:100690000F93022D003011F0222404C00F9301E0CB
:1006A000202E0F91032D003009F03A940F919FBF37
:1006B00018959FB70F9300E905BF78940F9188951F
:0606C0009FBF189518957C
:00000001FF
